:020000040000FA
:06000000CDEF10F012002C
:06080000CDEF10F0120024
:020808001200DC
:020818001200CC
:02082A000000CC
:04082C00C70E8B1652
:100830009416270E89169216F16A0101476B4D6BCB
:100840004E6B010E486F416B426B4B6B4C6B516BA7
:10085000526B536B566F576B906B586B0301186B51
:10086000080E185D1EE21851EA6A700FE96E010E5B
:10087000EA22EF6A1851EA6A780FE96E010EEA225D
:10088000EF6A1851EA6A910FE96E010EEA22EF6AE7
:100890001851EA6A990FE96E010EEA22EF6A182BE5
:1008A000DFD701015D6B5E6B5F6B596B5A6B5B6BE6
:1008B0005C6B8B6A896A970ED56EF50ECD6EB10EA4
:1008C000B16EA192170ECA6EFA0ECB6ECC6A9E92D2
:1008D000A16BA26BA36BA46BA56B120081CF19F364
:1008E0000101A1510301195D02E119C3A2F1A2C1E5
:1008F0001AF319C3A1F11A511200070E8014080D42
:10090000C70E8214F31003011B6F0101A3510301F1
:100910001B5D02E11BC3A4F1A4C11CF31BC3A3F123
:100920001C511200B2CF1DF3B35003011E6F1F6B99
:10093000176E166A1D511624146E000E172014C06F
:10094000F3FFF46E1200B2CF24F3B3500301256F0E
:10095000266B156E146A24511424226F000E152084
:10096000236F2251205D2351215906E22051225D3F
:10097000146E235121550DD020C316F021C317F05A
:10098000FF0ED8801656175616502225146E175093
:100990002321156E14C0F3FFF46E1200CC6A9E92F0
:1009A00012000101A5050DE1020E086E096A27C3B8
:1009B0000DF028C30EF097EC10F006C027F307C027
:1009C00028F327C314F028C315F0020E0F0B05E01F
:1009D000D89015321432E806FBE103012951EA6A86
:1009E000990FE96E010EEA2214C0EFFF27C35EF1F2
:1009F00028C35FF12A6B300ED8802755000E28558A
:100A000007E2900E275D000E285902E2010E53D036
:100A1000900E275D000E285907E3F00E275D000EAB
:100A2000285902E2020E47D0F00E275D000E285929
:100A300007E3500E275D010E285902E2030E3BD05A
:100A4000500E275D010E285907E3B00E275D010EF9
:100A5000285902E2040E2FD0B00E275D010E28594E
:100A600007E3100E275D020E285902E2050E23D07F
:100A7000100E275D020E285907E3700E275D020E47
:100A8000285902E2060E17D0700E275D020E285973
:100A900007E3D00E275D020E285902E2070E0BD0A5
:100AA000D00E275D020E285907E3300E275D030E96
:100AB000285902E2080E2A6F2A51000860E2DBDAA8
:100AC00001014D51070DF3CFE9FFF4CFEAFF000E0E
:100AD000E926020EEA2248C1EFFF4D51070DF3CF80
:100AE000E9FFF4CFEAFF000EE926020EEA22030E28
:100AF000E926000EEA2249C1EEFF4AC1EDFF4D5141
:100B0000070DF3CFE9FFF4CFEAFF000EE926020E4E
:100B1000EA22050EE926000EEA224BC1EEFF4CC187
:100B2000EDFF03012929100DF3502A25E66E01017E
:100B30004D51070DF3CFE9FFF4CFEAFF000EE92690
:100B4000020EEA22020EE926000EEA22E552E750E2
:100B5000EF6E4DC14FF14D2B280E4D5D01E34D6BF6
:100B60004E514D5D07E14FC14DF1080E516F050E1D
:100B7000526F536F482B485102E1010E486F030139
:100B80002A5112002BC3E9FF2CC3EAFFEF500408DF
:100B900006E1030E2BC3E9FF2CC3EAFFEF6E03014E
:100BA0002F0534E12BC3E9FF2CC3EAFFEF5008E126
:100BB000010E2BC3E9FF2CC3EAFFEF6ECEEF04F06A
:100BC0002BC3E9FF2CC3EAFFEF50020836E130C324
:100BD00029F32DC3E9FF2EC3EAFFEECF20F3EDCFBB
:100BE00021F3B1DEF3CF27F3F4CF28F3DADE0008E8
:100BF00007E2030E2BC3E9FF2CC3EAFFEF6E1200DE
:100C00002BC3E9FF2CC3EAFFEF6A12002BC3E9FFF5
:100C10002CC3EAFFEF0411E1020E2BC3E9FF2CC342
:100C2000EAFFEF6E7FDEF4CF15F02DC3E9FF2EC390
:100C3000EAFFF3CFEEFF15C0EDFF120031C3E9FF6D
:100C400032C3EAFFEF50040806E1030E31C3E9FFA7
:100C500032C3EAFFEF6E030135510EE131C3E9FF04
:100C600032C3EAFFEF5045E1010E31C3E9FF32C361
:100C7000EAFFEF6ECEEF04F031C3E9FF32C3EAFFC3
:100C8000EF0412E1020E31C3E9FF32C3EAFFEF6E57
:100C900049DEF4CF15F033C3E9FF34C3EAFFF3CFE5
:100CA000EEFF15C0EDFF120031C3E9FF32C3EAFFCA
:100CB000EF5002081EE136C329F333C3E9FF34C302
:100CC000EAFFEECF20F3EDCF21F33DDEF3CF27F3A4
:100CD000F4CF28F366DE000807E2030E31C3E9FF14
:100CE00032C3EAFFEF6E120031C3E9FF32C3EAFFFD
:100CF000EF6A12000101A5050EE13CC330F33BC3CE
:100D00002FF339C32DF33AC32EF337C32BF338C374
:100D10002CF3C2EF05F03CC336F33BC335F339C3C4
:100D200033F33AC334F337C331F338C332F31EEF2E
:100D300006F034DE0301406B0301405101E064D151
:100D400081CF3FF33F510101585D01E155D1010EC3
:100D500003013F15146E010E01015815145C20E0CB
:100D6000010E03013F15000809E2010E01015815AB
:100D700005E103013C6B03013B6B05D003013C6BB8
:100D80000301010E3B6F0301600E396F010E3A6FD4
:100D90000301700E376F010E386FACDF0101912B2C
:100DA000020E03013F15146E020E01015815145C6A
:100DB00021E0020E03013F1500080AE2020E0101C4
:100DC000581506E10301010E3C6F03013B6B05D092
:100DD0000301010E3C6F03013B6F0301620E396F8B
:100DE000010E3A6F0301710E376F010E386F82DF0B
:100DF0000101922B040E03013F15146E040E010134
:100E00005815145C22E0040E03013F1500080AE2A5
:100E1000040E0101581506E10301020E3C6F0301A7
:100E20003B6B06D00301020E3C6F0301010E3B6FCA
:100E30000301640E396F010E3A6F0301720E376FB2
:100E4000010E386F57DF0101932B080E03013F1588
:100E5000146E080E01015815145C22E0080E0301FF
:100E60003F1500080AE2080E0101581506E10301CA
:100E7000030E3C6F03013B6B06D00301030E3C6F76
:100E80000301010E3B6F0301660E396F010E3A6FCD
:100E90000301730E376F010E386F2CDF0101942BA5
:100EA000100E03013F15146E100E01015815145C4D
:100EB00022E0100E03013F1500080AE2100E0101A6
:100EC000581506E10301040E3C6F03013B6B06D08D
:100ED0000301040E3C6F0301010E3B6F0301680E1A
:100EE000396F010E3A6F0301740E376F010E386FC0
:100EF00001DF0101952B200E03013F15146E200E1A
:100F000001015815145C22E0200E03013F15000872
:100F10000AE2200E0101581506E10301050E3C6F9F
:100F200003013B6B06D00301050E3C6F0301010E6C
:100F30003B6F03016A0E396F010E3A6F0301750EA4
:100F4000376F010E386FD6DE0101962B400E03017C
:100F50003F15146E400E01015815145C22E0400E3E
:100F600003013F1500080AE2400E0101581506E191
:100F70000301060E3C6F03013B6B06D00301060E16
:100F80003C6F0301010E3B6F03016C0E396F010EC4
:100F90003A6F0301760E376F010E386FABDE010139
:100FA000972B800E03013F15146E800E010158151A
:100FB000145C22E0800E03013F1500080AE2800E57
:100FC0000101581506E10301070E3C6F03013B6B5D
:100FD00006D00301070E3C6F0301010E3B6F0301B6
:100FE0006E0E396F010E3A6F0301770E376F010EE7
:100FF000386F80DE0101982B3FC358F19EA29CD62A
:101000000301010E406F98D612000301436B080ED6
:10101000435D13E24351EA6A700FE96E010EEA2262
:10102000EF50030808E14351EA6A700FE96E010EC0
:10103000EA22040EEF6E432BEAD774DCF3CF3DF3C4
:10104000F4CF3EF376DE0301436B080E435D12E2FC
:101050004351EA6A700FE96E010EEA22EF5003086D
:1010600007E04351EA6A700FE96E010EEA22EF6A67
:10107000432BEBD712000101560525E1D6CF44F3EF
:10108000D7CF45F3F2A408D0F2944B2B000E4C239B
:10109000D6CF44F3D7CF45F3575107E17F0E030175
:1010A000455D02E2898601D0899603014551156AA2
:1010B00045C315F0146A445101011424496F000E10
:1010C00015204A6F1200D6CF44F3D7CF45F3030162
:1010D0004551156A45C315F0146A445101011424A1
:1010E000496F000E15204A6FF2A43CD0F2944B2BAE
:1010F000000E4C23D6CF44F3D7CF45F3030145511F
:10110000156A45C315F0146A445101011424496F4E
:10111000000E15204A6F575125E180BA1BD0000EF2
:10112000D8804955000E4A551DE24907000E4A5B1A
:1011300049C115F0146A1450151002E1000E01D0D7
:10114000010ED76E49514A1102E1000E01D0010E85
:10115000D66E1200492B000E4A23146A1450D76E23
:101160004951D66E1200060E0101CA5D01E29BD004
:101170006D50020B01E0120001019051000801E2E4
:1011800044DF79DF0101905176E16EEC04F001015A
:10119000596F7DEC04F001015A6F5B51595D03E119
:1011A0005C515A5D6CE059C15BF15AC15CF14D5123
:1011B000070DF3CFE9FFF4CFEAFF000EE926020E98
:1011C000EA2248C1EFFF4D51070DF3CFE9FFF4CFFD
:1011D000EAFF000EE926020EEA22030EE926000EBF
:1011E000EA2249C1EEFF4AC1EDFF4D51070DF3CF91
:1011F000E9FFF4CFEAFF000EE926020EEA22050E0F
:10120000E926000EEA224BC1EEFF4CC1EDFF4D5125
:10121000070DF3CFE9FFF4CFEAFF000EE926020E37
:10122000EA22020EE926000EEA2259C1EFFF4D51D3
:10123000070DF3CFE9FFF4CFEAFF000EE926020E17
:10124000EA22EE525AC1EFFF4DC14FF14D2B280E4D
:101250004D5D01E34D6B4E514D5D07E14FC14DF1C9
:10126000080E516F050E526F536F482B485107E11E
:10127000010E486F04D06EEC04F00101596F14D8D0
:101280009EA011D09E900101525100080BE252071E
:10129000525109E151075151000802E253C152F184
:1012A0006FEF0CF01CDB12000101400EC46F010156
:1012B000010EC26F010EC36FEBEC0FF0000901E1EC
:1012C000FDD20101006B01010151FF0A01E1E4D2ED
:1012D000BC0A01E1DBD2020A01E1B0D2010A01E15C
:1012E0008DD27F0A01E158D2040A01E148D2790A7D
:1012F00001E13ED2780A01E135D2030A01E107D2C9
:10130000010A01E1F6D10F0A01E1EBD1010A01E185
:10131000E0D1030A01E1C0D1010A01E1B5D10A0A15
:101320004FE00D0A4DE00F0A3FE00E0A2EE00F0AD3
:101330001FE00C0A0DE0310A01E0B0D20101040EF9
:10134000036F0101050E046F0101040E006FA7D2A7
:101350000101010E006FC70E010102158B6E380EE0
:1013600001010215E840E840E8401F0B896E97D262
:101370000101010E576F01010251E8B08986E8A012
:1013800089960101010E006F8AD20101020E006FE1
:101390006EEC04F00101026F7DEC04F00101036FBB
:1013A0000101030E006F7BD20101020E006F80BAB3
:1013B00003D00101026B03D00101010E026F6FD255
:1013C00003014C6B01014D5101014E5D01E1F9D06A
:1013D00001014E51070DF3CFE9FFF4CFEAFF000EF4
:1013E000E926020EEA22EF50E66E03014C51070D8A
:1013F000F3CFE9FFF4CFEAFF020EE926010EEA225D
:10140000E552E750EF6E01014E51070DF3CFE9FFB2
:10141000F4CFEAFF000EE926020EEA22030EE926C7
:10142000000EEA22EECF14F0EFCF15F003014C517D
:10143000070DF3CFE9FFF4CFEAFF020EE926010E14
:10144000EA22030EE926000EEA2214C0EEFF15C0C0
:10145000EDFF01014E51070DF3CFE9FFF4CFEAFF95
:10146000000EE926020EEA22050EE926000EEA2207
:10147000EECF14F0EFCF15F003014C51070DF3CF71
:10148000E9FFF4CFEAFF020EE926010EEA22050E7B
:10149000E926000EEA2214C0EEFF15C0EDFF01019F
:1014A00090514EE101014E51070DF3CFE9FFF4CF0A
:1014B000EAFF000EE926020EEA22020EE926000EDD
:1014C000EA22EF50E66E03014C51070DF3CFE9FF1E
:1014D000F4CFEAFF020EE926010EEA22020EE92607
:1014E000000EEA22E552E750EF6E03014C51070D62
:1014F000F3CFE9FFF4CFEAFF020EE926010EEA225C
:10150000EE52EF6A01014E51070DF3CFE9FFF4CF20
:10151000EAFF000EE926020EEA22EE52EF50E66ED6
:1015200003014C51070DF3CFE9FFF4CFEAFF020EA0
:10153000E926010EEA22EE52E552E750EF6E31D075
:1015400003014C51070DF3CFE9FFF4CFEAFF020E80
:10155000E926010EEA22020EE926000EEA2259C10E
:10156000EFFF01014E51070DF3CFE9FFF4CFEAFF82
:10157000000EE926020EEA22020EE926000EEA22F9
:10158000EF50E66E03014C51070DF3CFE9FFF4CFA6
:10159000EAFF020EE926010EEA22EE52E552E7507A
:1015A000EF6E03014C2B01014E2B280E01014E5D05
:1015B00002E301014E6B060E03014C5D01E101D017
:1015C00001D7060E03014C5D53E203014C51070D98
:1015D000F3CFE9FFF4CFEAFF020EE926010EEA227B
:1015E000EF6A03014C51070DF3CFE9FFF4CFEAFF97
:1015F000020EE926010EEA22030EE926000EEA2277
:1016000049C1EEFF4AC1EDFF03014C51070DF3CF75
:10161000E9FFF4CFEAFF020EE926010EEA22050EE9
:10162000E926000EEA224BC1EEFF4CC1EDFF03019B
:101630004C51070DF3CFE9FFF4CFEAFF020EE92684
:10164000010EEA22020EE926000EEA2259C1EFFF3E
:1016500003014C51070DF3CFE9FFF4CFEAFF020E6F
:10166000E926010EEA22EE525AC1EFFF03014C2B8C
:1016700003014C51070DF3CF14F0F4CF15F0010E18
:1016800014240101006F0BD15EC102F15FC103F1AF
:101690000101030E006F03D10101416B426BCECFFC
:1016A0004AF3CFCF4BF303014B51146E156A14C0AC
:1016B00015F0146A03014A5101011424456F000E0C
:1016C0001520466F0101010E476F0101010E006FE9
:1016D000E6D041C102F142C103F10101030E006FE6
:1016E000DED089860101010E576F0101010E006FE6
:1016F000D6D08996E4D80101010E566F0101576BCF
:101700000101010E506F0101010E006FC8D00101EF
:10171000506B0101546B80AA1CD00101010E506F67
:10172000F2A416D0F2940101545103080FE2010112
:10173000506B0101576B01010C0E516F0101080E36
:10174000526F0101080E536F04D002D00101542BD7
:10175000E2D7B5D80101020E566F0101576B0101A6
:10176000006B9DD050C102F10101020E006F97D0B5
:101770000101050E026F0101020E006F90D0010100
:101780000C0E516F0101080E526F0101080E536FCC
:101790000101010E006F83D002C190F10101586B6D
:1017A00003014D6B080E03014D5D13E203014D5122
:1017B000EA6A700FE96E010EEA22EF6A03014D51E9
:1017C000EA6A780FE96E010EEA22EF6A03014D2BF7
:1017D000E9D70101596B01015A6B01015D6B0101F0
:1017E0005B6B01015C6B01015E6B5F6B01014D6B1B
:1017F00001014E6B0101010E006F51D003014D6BD1
:10180000080E03014D5D16E203014D51EA6A910F86
:10181000E96E010EEA22EF50E66E03014D51EA6ACD
:10182000020FE96E010EEA22E552E750EF6E030166
:101830004D2BE6D70101090E006F31D003014D6B2E
:10184000080E03014D5D1EE203014D51EA6A990F36
:10185000E96E010EEA22EF50E66E03014D51EA6A8D
:10186000020FE96E010EEA22E552E750EF6E030126
:101870004D51EA6A990FE96E010EEA22EF6A0301FF
:101880004D2BDED70101090E006F09D002C1A5F171
:101890000101010E006F03D0FF0001D000D0010153
:1018A00000510CE004010CBF09D000C1C0F10101DE
:1018B000010EBE6F010EBF6FC5EC0FF01200F29467
:1018C000D76AD66AD76AF29401014B6B4C6B496BAD
:1018D0004A6B4E6B4EC14DF1010E486F120089A844
:0A18E00002D08998120089881200D6
:0618EA0004011851600B1F
:1018F000E842E842E842E842E842000901E012001A
:101900001951070A4CE00B0A4AE0070A3BE0010ABA
:1019100027E00B0A23E0020A21E0030A1DE0080A7F
:1019200012E0010A0EE00F0A0AE0030A01E01200C9
:101930000101010EA76F0101040ECA6F1200D0EF62
:101940000CF027EF0DF00101010EA76F0101CC0E85
:10195000A86F010EA96F10D04CEF0DF097EF0DF0AE
:101960000101010EA76F04011C510101A86FA96BB1
:10197000CD0EA827010EA9230101CB930101010E71
:10198000AC6F12000101010EA76F04011C51EA6A3D
:10199000CD0FE96E010EEA221AC4EFFF1200120009
:1019A000800E0401185D52E11B51030A30E0010A68
:1019B0000CE0030A49E10101010EA76F0101CE0EFF
:1019C000A86F200EA96F120E3CD00101010EA76F67
:1019D00004011A51F66EF76AD890F636F736240EDF
:1019E000F626210EF7220900F5CFA8F10A00F5CF5F
:1019F000A9F1020E0101F76AA825F66EA951F72296
:101A00000900F5CFACF10A00F5CFADF11DD0010111
:101A1000010EA76F04011A51F66EF76AD890F636D8
:101A2000F736280EF626210EF7220900F5CFA8F189
:101A30000A00F5CFA9F1A8C1F6FFA9C1F7FF080078
:101A4000F5500101AC6FAD6B0101CB8312000101B8
:101A5000010EA76F01010F0EC96F0101710EC76F53
:101A60000F0EC86FA4EC0FF00101010EC96F010148
:101A7000CD0EC76F010EC86FA4EC0FF01AC4CCF1E5
:101A800004011A5104E10101050ECA6F120001019F
:101A9000060ECA6FB0EF0FF00401206B216B04013A
:101AA00018511F0B020A13E0030A0DE0010A31E18D
:101AB0000101010EA76F040120810101CBA129D0F2
:101AC0000401208326D00101010EA76F22D001015D
:101AD000010EA76F04011C510F0B080DF350156A7E
:101AE000000F146E040E15221C51800B01E0010E34
:101AF000040DF35001011424AA6F000E1520AB6FE2
:101B0000AAC1E9FFEA6EEF50040B03E00401010EE5
:101B1000206F0101A7050AE10101200EA86F040E44
:101B2000A96F0101CB930101020EAC6F12000401F9
:101B30001A0510E118511F0B00090CE10101010EFB
:101B4000A76F030E0401195D03E10101CB8102D0EF
:101B50000101CB9104011A513AE118511F0B0208FF
:101B600036E11C510F0B000932E00101010EA76F95
:101B700004011C510F0B080DF350156A000F146E71
:101B8000040E15221C51800B01E0010E040DF350D0
:101B900001011424AA6F000E1520AB6F030E04017F
:101BA000195D07E1840EAAC1E9FFABC1EAFFEF6E40
:101BB00012001CAF06D0AAC1E9FFABC1EAFFEF6A71
:101BC0001200880EAAC1E9FFABC1EAFFEF6E120056
:101BD0006C5002E0000E01D0010E00090BE0040180
:101BE00000513C0BE842E8420D0802E103EF0EF021
:101BF0000CEF0EF06C5002E0000E01D0010E040953
:101C000001E019D812000101A66BA76BAC6BAD6B9C
:101C100075EC0CF0B0EF0EF0020E0101A65D09E1CB
:101C200078D8040100BD02D0C80E01D0880E006F24
:101C30001200F5EF0EF0040E0101CA5D09E11AC4AD
:101C40006EFF6E50000802E2050E01D0030ECA6F4F
:101C50000101A60509E10AD8040104BD02D0C80E9D
:101C600001D0880E046F1200F5EF0EF00101080E8E
:101C7000AC5D000EAD5905E2ACC1AFF1ADC1B0F144
:101C800003D0080EAF6FB06B0401049304910101FF
:101C9000B05104010413AFC105F40101AF51AC5DB3
:101CA000AC6FB051AD59AD6F200EAA6F040EAB6F83
:101CB0000101CBA317D00101AF51B01129E0A8C198
:101CC000F6FFA9C1F7FF0800F550AAC1E9FFABC1B3
:101CD000EAFFEF6EAA2B000EAB23A82BA923AF07B8
:101CE000B05BE9D70101AF51B01112E0A8C1E9FF23
:101CF000A9C1EAFFEF50AAC1E9FFABC1EAFFEF6E4D
:101D0000AA2B000EAB23A82BA923AF07B05BEAD701
:101D10001200030E040100150101B26F01C4B1F1FC
:101D2000AC51B125AC6FAD51B221AD6F200EA86F93
:101D3000040EA96FB151B21112E0A8C1E9FFA9C107
:101D4000EAFFEF50AAC1E9FFABC1EAFFEF6EAA2B91
:101D5000000EAB23A82BA923B107B25BEBD712006F
:101D60000101A7510BE10401080E016F180E026F6B
:101D7000040E036F840E006F040123D0040118AF1A
:101D800022D00101AC5104011E5D0101AD510401DD
:101D90001F5904E21EC4ACF11FC4ADF167DF01019D
:101DA000010EA66F0401080E016F180E026F040EDB
:101DB000036F800E006F0401200E066F040E076F84
:101DC000C80E046F10D00101020EA66F0401056B4E
:101DD000C80E046F0401080E016F200E026F040E7E
:101DE000036FC80E006F6D9812000101A66B04010D
:101DF000080E016F180E026F040E036F880E006F3D
:061E00000401046B120056
:0A1E06006DA60CD80101CA0508E121
:101E10006DBA06D0686A696A69806988020ECA6FFD
:101E200012006D6A696A6D860101010ECA6F1200A7
:101E30006D6A696A0101CA6B120018EF0FF00101A7
:101E4000CA5101E112006850040B04E06950040B10
:101E500001E038D86DB212006850010B04E06950FF
:101E6000010B01E050D86850100B04E06950100BD2
:101E700001E024D86850400B04E06950400B01E0B9
:101E800037D86850200B04E06950200B01E032D8AD
:101E90006850020B04E06950020B01E032D8030ED7
:101EA0000101CA5D01E212006850080B06E06950AA
:101EB000080B03E0E8EC0DF068961200698468985E
:101EC0006D8212006D926994689412000101CBA199
:101ED0000ED0F8DF6D840101080EC56F070EC66FC6
:101EE000C507000EC65BC551C611FAE16D9412001C
:101EF000689C120070A003D0F5EC0EF07090689A08
:101F00001200689212006A6A686A9F0E6B6E7B0EFE
:101F1000696E6E6A01010F0EC96F0101710EC76F04
:101F20000F0EC86F11D8160E706E68A602D0689694
:101F3000FCD76D98F5EC0EF00101CB910101CC6B53
:101F40000101030ECA6F1200C7C1E9FFC8C1EAFF51
:101F50000101C95104E0EE6A0101C907F9D7120075
:101F60000101BD6B1E0E716E0401400E096F280E3B
:101F70000A6F040E0B6F880E086F0401680E0E6F57
:101F8000040E0F6F400E0C6F12000101C05140088B
:101F900002E2400EC06FC16BC051C15D13E2C1517E
:101FA000EA6ABE25E96EBF51EA22EF50E66EC151E2
:101FB000EA6A680FE96E040EEA22E552E750EF6E16
:101FC000C12BEAD7C0C10DF4400E04010C170C7DE3
:101FD000880E0C1312000101BD6B040108BF25D04F
:101FE00009510101D880C45502E209C4C4F1BD6B96
:101FF000C451BD5D13E2BD51EA6A280FE96E040EBB
:10200000EA22EF50E66EBD51EA6AC225E96EC3517D
:10201000EA22E552E750EF6EBD2BEAD70401400EED
:10202000096F0817087D880E08130101BD511200C1
:102030002A0EF66E080EF76E000EF86E010109000A
:10204000F550B86F0900F550B96F03E1B86701D0DA
:102050003DD00900F550B36F0900F550B46F090089
:10206000F550B56F09000900F550E96E0900F5500B
:10207000EA6E090009000900F550B66F0900F55035
:10208000B76F09000900F6CFBAF1F7CFBBF1F8CF6F
:10209000BCF1B3C1F6FFB4C1F7FFB5C1F8FF010150
:1020A000B65302E1B75307E00900F550EE6EB607EC
:1020B000F8E2B707F9D7BAC1F6FFBBC1F7FFBCC159
:0E20C000F8FF0101B807000EB95BBFD7120090
:0220CE001201FD
:1020D000000200000008D804010F00000102000106
:1020E0000902200001010080320904000002000002
:1020F0000000070501034000200705810340002080
:1021000004030904100343006F0063006B007000B8
:102110006900740010035500530042002D00420076
:0E2120006F007800E020E0200021042114214F
:02212E0008C0E7
:1021300012F008500D02F4CF07F0F3CF06F009506B
:102140000E02F4CF09F0F3CF08F00D02F35007268A
:10215000F4500822E86A092212500E02F3500726B2
:0A216000F4500822E86A0922000C7E
:06216A0004D80FD8B3EC0D
:1021700008F0FCD70F0EC112140E6F6E0101CA6B6E
:102180000101CB6B0101CC6B16EF04F003EC0FF0F7
:0A2190006FBE02D01FEC0FF012002A
:06219A0013EE50F023EEED
:1021A00050F0F86A019C18EC10F0DBEC10F0B5EC84
:0621B00010F0FBD7120045
:0221B600120015
:00000001FF
